:100000000EC028C078C126C025C024C023C022C08D
:1000100021C020C0CFC11EC01DC01CC01BC01124E8
:100020001FBECFE5D1E0DEBFCDBF10E0A0E6B0E05F
:10003000EEE0F8E002C005900D92AC39B107D9F7B7
:1000400010E0ACE9B0E001C01D92AB3AB107E1F7B6
:10005000E1D2DBC3D5CFDF93CF930F92CDB7DEB71D
:1000600082E389838981982F915099838823D1F7DE
:100070000F90CF91DF91089590E087FF02C0C19A61
:1000800001C0C198C29A9F5FC298983011F0880F42
:10009000F4CF0895DF93CF930F92CDB7DEB7C09A18
:1000A00082E389838981982F915099838823D1F79E
:1000B000C0980F90CF91DF9108951092A6001092F2
:1000C000A7001092A8001092A900089587B3876036
:1000D00087BB1092A6001092A7001092A800109261
:1000E000A90080E0C9DF8091A700C6DF8091A80049
:1000F000C3DF8091A900C0DFCDDF08956F927F92AA
:100100008F929F92AF92BF92CF92DF92EF92FF9227
:100110000F931F93DF93CF93CDB7DEB7AC970FB696
:10012000F894DEBF0FBECDBFFA01AE014F5F5F4F47
:1001300000E710E02CE2D8010D908D01DA010D925C
:10014000AD012150C1F7611571058105910509F4D3
:100150004FC097FF09C090958095709561957F4F2E
:100160008F4F9F4F2DE22193DE01119620E001C0B9
:100170002F5FED90FD900D911D916E157F0580070D
:100180009107B0F3332727FD3095220F331F220F3D
:10019000331FDE011196A20FB31FED90FD900D915C
:1001A0001C911397E114F1040105110519F166245E
:1001B000772443016E187F08800A910A5B016C0165
:1001C000AE18BF08C00AD10A20E3C601B501D7FEA8
:1001D00005C06E0D7F1D801F911F07C02F5FA60CED
:1001E000B71CC81CD91C2A3381F721931496D5CF8C
:1001F00080E381931082AC960FB6F894DEBF0FBEF9
:10020000CDBFCF91DF911F910F91FF90EF90DF90C5
:10021000CF90BF90AF909F908F907F906F900895F8
:1002200084E08093A6008093A7008093A800809329
:10023000A900089580E48093A6008093A70080938E
:10024000A8008093A900089521E02093A300909333
:10025000A5008093A4001092A30008951092AA0014
:100260008091AA008823E1F3089508C01092AA00A3
:100270002091AA002223E1F30197A8950097B1F7F6
:10028000089589B78F7E89BF20919F003091A0008B
:100290004091A1005091A20089B7806189BFB90146
:1002A000CA0108959B01AC0189B78F7E89BF209355
:1002B0009F003093A0004093A1005093A20089B703
:1002C000806189BF0895805787B9369A3699FECFE5
:1002D00024B135B1C9010895F89488E181BD8FE05A
:1002E00081BD78940895F894A89514BE88E181BDE5
:1002F00011BC789408951F920F920FB60F9211249B
:100300008F939F93DF93CF930F92CDB7DEB7AC98C7
:10031000B49B0BC0C49ABC9A82E389838981982FCD
:10032000915099838823D1F70DC081E080939D007F
:10033000C498BC9A82E389838981982F91509983CC
:100340008823D1F7BC98C49A80E28ABFAC9A0F90F8
:10035000CF91DF919F918F910F900FBE0F901F90C3
:10036000189587E886B9089581E08093A30081E01D
:1003700090E09093A5008093A4001092A3001092A7
:100380009F001092A0001092A1001092A200109263
:10039000AA0082E08ABD8CE989BD83E083BF80E149
:1003A00088BF89B7806189BF87E886B9089519BE7B
:1003B00016B808951F920F920FB60F9211241F9333
:1003C0002F933F934F935F936F937F938F939F935D
:1003D000AF93BF93EF93FF9310919C008091A9007E
:1003E00081274ADE8091A800812746DE8091A70000
:1003F000812742DE8091A60081273EDEC09A1095BB
:1004000010939C0021E02093AA0080919F0090917E
:10041000A000A091A100B091A2000196A11DB11D64
:1004200080939F009093A000A093A100B093A2009E
:10043000C0988091A300882391F48091A4009091AA
:10044000A500009719F42093A30009C08091A4008F
:100450009091A50001979093A5008093A400FF912F
:10046000EF91BF91AF919F918F917F916F915F912C
:100470004F913F912F911F910F900FBE0F901F90A2
:100480001895EF92FF920F931F93DF93CF93CDB701
:10049000DEB72F970FB6F894DEBF0FBECDBF683A18
:1004A00021EC720720EF82072FEF920714F480E40B
:1004B00009C06939E2E97E07E8E98E07E0E09E07B6
:1004C00054F084E08093A6008093A7008093A80056
:1004D0008093A90092C09B01AC01222757FD239570
:1004E000332744275527F22E8E010F5F1F4FA80197
:1004F00005DED8010D900020E9F7119740E050E0AB
:10050000A01BB801BA2FBF5F2F2D332727FD3095D1
:10051000200F311F90E312C08B0FE82FFF27E7FD5C
:10052000F095E60FF71F04C0E080E182815031971B
:100530008F15D4F7F90190834F5F5F4F842FE42F1D
:10054000EA0FE4304CF3F80101900020E9F731970D
:10055000E01BF10B2E2F2F5F332727FD3095DB019A
:10056000A20FB31F80E090E0A901FF27E7FDF095FF
:10057000339706C02C9111962C93119701971197E0
:100580009C01240F351F2E173F07A4F72C0F3D1F8A
:100590008EE2F9018283E6EAF0E080E09E012F5FBF
:1005A0003F4F41E0A82FBB27A7FDB095A20FB31F77
:1005B000AC91AD3211F4408319C0AE3281F48F5F3B
:1005C000A82FBB27A7FDB095A20FB31FAC91BB27E7
:1005D000A7FDB095A05DBF4F9C91905F06C0BB2763
:1005E000A7FDB095A05DBF4F9C919083319690E0A0
:1005F000EA3AF90711F08F5FD5CF2F960FB6F8942E
:10060000DEBF0FBECDBFCF91DF911F910F91FF9045
:10061000EF9008956F927F928F929F92AF92BF92C8
:10062000CF92DF92EF92FF920F931F93DF93CF93BE
:100630000F92CDB7DEB780E886BD83E086BDAC9A69
:1006400080E28ABF8BB780628BBF40DDF89488E17F
:1006500081BD8FE081BD789487DE7894C49A8AE06A
:1006600090E003DE81E080939D00B49902C0809306
:100670009E0000E3C02E18E1D12EBFE0EB2EFF2438
:10068000F394A1E26A2E712C00E217E880919D009C
:100690008823B1F028DE19BE16B818DD80919E00BF
:1006A000882321F4B49BFECFC5BE889510929D008F
:1006B00010929E000BDDF894D1BCE1BC789454DE1E
:1006C000F092A3007092A5006092A4001092A30083
:1006D00088249924540120E083E02983F4DDA0E0FC
:1006E000B0E0880E991EAA1EBB1E29812F5F2A30FA
:1006F00099F7C501B401F2E09595879577956795CF
:10070000FA95D1F7BEDE16B803C0A89505BF889547
:100710008091A3008823C9F316B9B8CF0F931F9314
:10072000DF93CF93CDB7DEB72F970FB6F894DEBF28
:100730000FBECDBF611571058105910549F4109279
:10074000A6001092A7001092A8008091600019C026
:1007500069312CEF72072FEF82072FEF920714F405
:1007600080E409C06031A7E27A07A0E08A07A0E030
:100770009A0754F084E08093A6008093A7008093AA
:10078000A8008093A90036C08E010F5F1F4FA801FB
:10079000B5DCD8010D900020E9F71197A01BB10B33
:1007A00080E090E005C0FC01EA55FF4F1082019601
:1007B000E82F282F2A0F2430B4F3AE014F5F5F4F8C
:1007C000FF27E7FDF095EA55FF4F21E00FC08D327E
:1007D00011F4208308C0992787FD9095805D9F4F75
:1007E000DC018C9180834F5F5F4F3196DA018C91F1
:1007F000882369F72F960FB6F894DEBF0FBECDBFE2
:0E080000CF91DF911F910F910895F894FFCFD3
:10080E00EE886DCD8BC7E78CEFCFAFE366E9672738
:10081E0000CA9A3B00E1F5058096980040420F0011
:10082E00A086010010270000E8030000640000000D
:0C083E000A0000000100000000000000A3
:00000001FF
